:0C0000000C9469000C9400000C940000AB
:10000C000C9400000C9400000C9400000C94000064
:10001C000C9400000C9400000C9400000C94000054
:10002C000C9400000C9400000C9400000C94000044
:10003C000C9400000C94CB000C9400000C949800D1
:10004C000C9400000C9400000C9400000C94000024
:10005C000C9400000C9400000C9400001027E80392
:10006C0064000A00010000100001100001000000F3
:10007C0000000A000000000000000000000000006A
:10008C000000000000000000000000000000000064
:10009C000000000000000000000000000000000054
:1000AC0000000A0A0A0A0A0A0A0A0A0A0A0A0A0AB8
:1000BC000A0A020002007A00020004007C0001001F
:1000CC0009037E000000F894EE27EFBBF1E0F5BFCA
:1000DC00E5BF8DE0A2E0BB27ED938A95E9F780E0C0
:1000EC0098E0A0E0B1E0ED930197E9F7EEEBF0E0DA
:1000FC0085919591009761F0A591B591059015901A
:10010C00BF01F00105900D920197E1F7FB01F0CFD3
:10011C00E8E0EEBBEFEFEDBFE8E0EEBFC0E0D3E010
:10012C000C944403AA93EA93FA93EFB7EA931A93C5
:10013C000A931091C0000091C600E12FEC71E9F414
:10014C00E091CC03EF5FE093CC03E150F0E0ED5491
:10015C00FC4F0083A091CC03A93119F4E0E0E093AB
:10016C00CC03A091CE03AF5FA093CE03A93129F4A9
:10017C00E0E0E093CE03689433F809911991E9918A
:10018C00EFBFF991E991A99118950A921A926A9385
:10019C007A938A939A93AA93BA93EA93FA93EFB7C2
:1001AC00EA93E0912B03F0912C033196E0932B030F
:1001BC00F0932C030E940D19E1E5F1E00E94C0219F
:1001CC000E2E0E940D19E3EAF2E00E94C021E029F4
:1001DC0009F4C3C1A0912903B0912A03E4E1F0E032
:1001EC000E94D2210E2EE0910603F0E074970E943B
:1001FC0012190E94C6210E22A0911803EEE00E9453
:10020C00B621E02121F0E0911803EF5F03C025FC3B
:10021C0003C0E0E0E0931803A0911803AE3011F492
:10022C00689425F8E0912903E0930603A091190343
:10023C00A13029F4F79B02C0F79801C0F79AE1E0CE
:10024C002E260E9417190E942019E0939B03F0930D
:10025C009C0360939D0370939E030E942719AFE744
:10026C00B3E00E942C190E943319ABEAB3E00E9450
:10027C002C190E9438190E9441190E94F120E09318
:10028C007F03F09380036093810370938203A091AA
:10029C00AB03B091AC038091AD039091AE03E0E061
:1002AC00F0E060E772E40E94F120E093AB03F0937E
:1002BC00AC036093AD037093AE030E9446190E9489
:1002CC004B190E2E0E9450190E944B19E02161F11E
:1002DC00E091AB03F091AC036091AD037091AE0370
:1002EC000E9438190E94F120E093A703F093A80311
:1002FC006093A9037093AA030E945519AFE3B3E06E
:10030C000E945E19A091A703B091A8038091A90344
:10031C009091AA030E942019E0938703F09388031D
:10032C006093890370938A030E946319E0E0F0E004
:10033C006AE774E40E946C190E9471190E945320A0
:10034C00E0938F03F0939003609391037093920367
:10035C000E947A190E947F190E949019A7E5B3E0B8
:10036C000E9495190E949A190E9463190E941920E3
:10037C000E946C19E0939F03F093A0036093A10378
:10038C007093A203A091AF03B091B0038091B1031D
:10039C009091B2030E945320E093AF03F093B0030B
:1003AC006093B1037093B2030E947A19E5E20E9444
:1003BC00A319A9E5B3E00E9495190E9417190E9490
:1003CC000A23DCF40E94B319A0E0B0E080E89FE3BC
:1003DC000E94F120A0919F03B091A0038091A103F2
:1003EC009091A2030E94A320E0939703F0939803AB
:1003FC006093990370939A0309C0E0E0E09397032C
:10040C00E0939803E0939903E0939A030E94BC193C
:10041C00AEE1B3E00E94E01FEC930E94B3190E947E
:10042C00C5190E9453200E94CE19E0917F03F091D0
:10043C00800360918103709182030E94D7190E94FE
:10044C00362168F5E0918703F09188036091890368
:10045C0070918A030E94D7190E945320E093830362
:10046C00F093840360938503709386030E94D719DD
:10047C000E94E0190E944C20DF01CB010E9455190B
:10048C000E94F120A0E0B0E081E695E40E94A32058
:10049C00A3E5B3E00E949519689424F802C0E0E14A
:1004AC002E260E94B3190E94E9190E945320E09352
:1004BC008B03F0938C0360938D0370938E030E94D7
:1004CC00E919E0E0F0E060E87FE30E94362109F0F2
:1004DC0008F416C0E0938B03E0938C03E0938D0338
:1004EC00E0938E030E94F219EF5FFF4F6F4F7F4F27
:1004FC000E94FB190E94F219A9E2B0E00E94DF22CF
:10050C000E94041AA034E2E4BE07EFE08E07E0E09C
:10051C009E0778F0E0E0E0934903E0934A03E09310
:10052C004B03E0934C03A9E2B0E00E940D1A0E9429
:10053C00DF220E94C5190E9441190E94A320ADE23E
:10054C00B3E00E945E19A0911603AC3308F4F29844
:10055C00A0911603AC3309F4F29A0E940D19A33A38
:10056C00E2E0BE0709F061C0A09115030E94121AC7
:10057C000E94171A0E940D1A0E94D8210E94201A5C
:10058C0091F0E0911603EF5FE0931603E0911503F1
:10059C00F0E03296A0911603B0E0EA17FB0719F4CD
:1005AC00ECE3E0931603E0E0E0932B03E0932C03E1
:1005BC00C394A0914303B0914403E8E5F2E00E9498
:1005CC00CC210E2E0E94281AE02199F0E0914303D1
:1005DC00F09144033196E0934303F09344030E945B
:1005EC00171A0E940A232CF4E0E0E0934303E093F3
:1005FC004403ECE3EC15C9F4CC24E0910003EF5F69
:10060C00E0930003A0910003AC3379F4E0E0E093B5
:10061C000003E0910103EF5FE0930103A09101035C
:10062C00A43119F4E0E0E0930103E991EFBFF991F3
:10063C00E991B991A99199918991799169911990BF
:10064C0009901895AA93E881E066E0937C0085E216
:10065C008A95F1F7E0917A00E064E0937A00E091FA
:10066C007A00E071E1F3E0917A00E061E0937A00C6
:10067C00E0917800F091790021960895EF972197F9
:10068C008EE3A2E0B0E0E0E8F0E00E941F23FF243C
:10069C0001E020E0E0E8E0936100E0E0E09361003D
:1006AC00EFE0E4B9E1E0E5B9E0E0E7B9E4E0E8B9AE
:1006BC00EAEFEAB9E7EEEBB9E0E0E4BDE3E0E5BD73
:1006CC00E0E0E6BDE7BDE8BDE1EAE0938000E2E0F2
:1006DC00E0938100E0E0E0938500E0938400E093F8
:1006EC008700E0938600E0938900E0938800E09314
:1006FC008B00E0938A00E093B600E1EAE093B0004F
:10070C00E2E0E093B100E0E0E093B200E093B300EC
:10071C00E093B400E1E0E0936E00E0E0E0936F0062
:10072C00E0937000E0936900EDBBE0936800E09308
:10073C00C000E8E9E093C100E6E0E093C200E0E02D
:10074C00E093C500E7E4E093C400E0E8E0BFE0E03C
:10075C00E0937F00E0937E00E0E6E0937C00E7E22C
:10076C00E0937A00E0E0E0937B00ECBDE093BC000A
:10077C0078940E942D1A0E94351A0E94421A0E94E7
:10078C004F1AEAE09E1630F4ABE1B0E0E0E0F0E0A6
:10079C000E94E722EAE08E1640F4A1E2B0E0E0E02D
:1007AC00F0E00E94E722689426F8EAE0AE1618F40E
:1007BC00689430F827F80E94591A0E94601A0E9417
:1007CC00671AE8ECF0E0E0934D03F0934E03EEE093
:1007DC00E0930A03A0E0B0E00E94D322E0930B0365
:1007EC00A1E0B0E00E94D322E0930C03A2E0B0E0C1
:1007FC000E94D322E0930D03A3E0B0E00E94D32229
:10080C00E0930F03A4E0B0E00E94D322EE8BA5E0AE
:10081C00B0E00E94D322EF8BA6E0B0E00E94D3227E
:10082C00E88FA7E0B0E00E94D322E0931003A8E089
:10083C00B0E00E94D322E0931103A9E0B0E00E9443
:10084C00D322E0931203F798F198AAE0B0E00E944B
:10085C00D322E0931503A9E1B0E00E94CF220E94BD
:10086C006E1AA4E1B0E00E94D322EA8BA5E1B0E0BD
:10087C000E94D322EB8BA6E1B0E00E94D322EC8B3A
:10088C00ABE0B0E00E94D322EE87ACE0B0E00E9477
:10089C00D322EF87ADE0B0E00E94D322E88BADE12C
:1008AC00B0E00E94CF22ED83FE83AEE0B0E00E9468
:1008BC00D322E0931A03AFE0B0E00E94D322E0937E
:1008CC001C03A0E1B0E00E94D322E0931B03A9E239
:1008DC00B0E00E94CB220E94FB19ABE1B0E00E9479
:1008EC00CF22ABE7B3E00E94731A0E94E019ADE28D
:1008FC00B3E00E945E190E94C5190E9441190E9422
:10090C00F1200E94CE19A1E1B0E00E94D3223E2F2B
:10091C00AFE1B0E00E94CF22E987FA87A2E1B0E014
:10092C000E94D322EA8FA3E1B0E00E94D322E98F88
:10093C00A1E2B0E00E94CF22AFE8B3E00E94731AAC
:10094C00A3E2B0E00E94CF220E947A1AA7E2B0E0A4
:10095C000E94CF220E947F1AA7E1B0E00E94D3220E
:10096C000E941A2323F8A5E2B0E00E94CF220E9435
:10097C00841AA8E1B0E00E94D322E0930803A0916E
:10098C000303A43128F4E0910303EF5FE093030326
:10099C00A0910303A431A1F4E0E0E0932003E093E1
:1009AC002103EBE0F0E0E0934703F0934803E8EB1E
:1009BC00E0932203E0E0E093CC03EAE0E09303034E
:1009CC00A091CC03AB30C1F4E091B603E0932003CB
:1009DC00E091B703E0932103E091B803F0E0E093DA
:1009EC004703F0934803E091B903E0932203E0E05E
:1009FC00E093CC03E0930303A091CC03AC30C0F0A4
:100A0C00E0E0E093B303E093B403E093B503E09329
:100A1C00B603E093B7030E94591AE0E0E093BA03DF
:100A2C00E093BB03E093BC03E093BD03E093CC03E2
:100A3C00E8EC5E1630F45394E4E1E51511F4E1E0D2
:100A4C004E2E0E942D1AA0E00E94891A3B9798F115
:100A5C00A0E00E948E1A662777270E94951A0E94A2
:100A6C009A19A8EEB3E080E090E00E942322DF0107
:100A7C00CB010E949E1A662777270E9465220E944E
:100A8C00951AE0910903EF5FE0930903E0910803E5
:100A9C00A0910903AE1768F00E949A19E0936B03BA
:100AAC00F0936C0360936D0370936E03E0E0E0933E
:100ABC000903E894F3F80E94A31A0E94351AA2E0E5
:100ACC000E948E1ADF01E5E0F0E00E942822BE2E83
:100ADC000E94A31A0E94421AA7E00E94891A0E943F
:100AEC00AA1A0E94A31AA5E00E94891A1E2F0E941E
:100AFC00A31AA0E00E94891ADE2E0E94A31A0E945B
:100B0C004F1AE7EAE0937A00A6E00E94891AEC8774
:100B1C00E7E2E0937A00E1E0E51591F50E94121905
:100B2C00E2E3F0E00E94D2210E2E0E94AF1A0E9446
:100B3C00CC21E02111F0E5E0EB87A12FE2E30E944C
:100B4C00BB210E2EEAEF0E94B621E02111F0E6E067
:100B5C00EB870E94AF1A0E94D2210E2E0E94B31A6C
:100B6C00E02911F0E7E0EB87A12FEAEF0E94BB210F
:100B7C000E2EEEE10E94B621E02911F0E8E0EB87A1
:100B8C000E94AF1A0E94D2210E94B91A39F0E1E0FA
:100B9C00EB87E8E2F0E00E94AA1A07C00E94B31AA1
:100BAC000E94B91A11F0E2E0EB87A12FEAEF0E9444
:100BBC00BB210E94B91A11F0E3E008C0A12FEEE1AD
:100BCC000E94B6210E94B91A19F0E4E0EB871CE3ED
:100BDC00AB850E94C51AAB85E7E00E94A2210E2AC4
:100BEC00E1E00E94A2210E2AE2E00E94A221E0296B
:100BFC0029F0E12FF0E00E94AA1A18E2AB850E94BE
:100C0C00CA1AAB85E8E00E94A221E02909F018E29B
:100C1C000E94CF1A0E94D51A0E94B621E021D1F071
:100C2C006894F3F8013021F4F398F49A02E012C0BE
:100C3C00023059F4F498F59AA88DA13010F003E025
:100C4C0003C0F598F39A01E005C0033019F4F59848
:100C5C00F39A01E00E941219D39708F457C00E942E
:100C6C00DF1A0E94E41AE02F0E94EB1A20F0E8EC45
:100C7C00F0E00E94AA1AE02F0E94FB1A0E940B1BA4
:100C8C00AC91A13008F441C00E94121B0E941B1BA6
:100C9C000E9415234CF40E940B1B0E94271B0E94E0
:100CAC0062210E94321B23C00E943B1B0E943D1BF1
:100CBC00EF930E943B1B0E94461BAF91EA2379F0F5
:100CCC000E940B1B0E94271B0E946721A0935B03B1
:100CDC00B0935C0380935D0390935E0308C00E9405
:100CEC003B1B0E944F1B1CF00E94591B0EC0A09175
:100CFC005B03B0915C0380915D0390915E030E9455
:100D0C00611B0E9465220E94AA1A04C00E94661BE5
:100D1C000E94591B0E946C1B0E94721B0E220E9487
:100D2C00771BE02139F0E0912703E09317036894D7
:100D3C00F0F821F80E94DF1A309721F4E0E0E093FC
:100D4C00180306C0A0911803A23010F4E89425F8FB
:100D5C000E94DF1AE0932903F0932A030E94DF1A02
:100D6C00309719F4E89421F813C0A0E021FCA1E01D
:100D7C00E0E00E94A2210E2EA09117030E947E1B80
:100D8C0039F0E0E0E09317030E94661BE89422F828
:100D9C00A0911703A13040F0689422F8E09117035A
:100DAC00F0E00E94AA1A02C0E89422F8E091050330
:100DBC000E941219F0E0AE17BF0720F0E091270354
:100DCC00E0930503E0910503F0E035970E941219BA
:100DDC00AE17BF0770F4E0912703E093050325FEDF
:100DEC0008C0E2E0E0931D03E89425F8E0E0E0930E
:100DFC001803A0911D030E94121A0E94831B0E94CB
:100E0C00E8210E22A0911A030E948A1B1E2EA0918B
:100E1C001D030E94121A0E94831B0E94E0210E22C5
:100E2C00A0911B030E948A1BE12959F00E94121900
:100E3C001B9710F00E94661BE0911D03E150E0939C
:100E4C001D030E948F1B0E22A0E031FCA1E00E942A
:100E5C008A1B31F0689431F80E94DF1A0E94A51B9E
:100E6C000E948F1BE02161F10E94AA1B0E94B21B01
:100E7C00A4F0A0916703B0916803ED81FE81EA1B99
:100E8C00FB0BA3E0B0E00E941E220E94BA1BAE1B1B
:100E9C00BF0BA0934F03B09350030E94AA1B0E9458
:100EAC000A232CF40E94BF1B32970E94A51BA09111
:100EBC005003AA232AF4E0E0E0934F03E09350039D
:100ECC000E94C41B0E94102384F5E89431F80E9400
:100EDC00C41B0E9467210E94B21B74F0AD81BE81BD
:100EEC00E0916703F0916803EA1BFB0B0E94BA1BAD
:100EFC00EA0FFB1F0E94A51B0E94C41B0E946721C6
:100F0C00A230E0E0BE07E0E08E07E0E09E072CF0A8
:100F1C000E94BF1B31960E94A51B0E94BA1BA93CC4
:100F2C00E0E0BE0714F00E94601A0E94BF1B0E94F2
:100F3C001219EA17FB0720F40E94BF1B0E94AA1A81
:100F4C000E94D11B0E945C210E2EA0E032FCA1E07D
:100F5C000E948A1B59F0689432F80E941219EAE038
:100F6C000E941822E0935103F09352030E94D11B6C
:100F7C000E94362109F008F435C00E94E01BDF0105
:100F8C00CB01E0E0F0E060E070E40E94362109F073
:100F9C0008F410C00E94E01BDF01CB01E985FA8543
:100FAC000E94EF1B0E94F61B0E94FB1BA1E5B3E005
:100FBC000E9495190E94E01B0E94002354F4EA8DB4
:100FCC00F0E00E94F61BAE1BBF0BA0935103B09335
:100FDC005203A0915203AA232AF4E0E0E0935103B8
:100FEC00E09352030E94D11B0E943621F0F5E89445
:100FFC0032F80E94001CDF01CB01E0E0F0E060E47D
:10100C0070E40E94362109F008F418C00E94001CFC
:10101C00A0E0B0E080EA90E40E94A320DF01CB01C5
:10102C00E0915103F09152030E9498210E941920E3
:10103C000E945320A1E5B3E00E9495190E94001C68
:10104C000E94002354F4E98DF0E00E94F61BEA0F95
:10105C00FB1FE0935103F09352030E94F61BA13D3A
:10106C00E7E0BE0714F00E94671A0E941219EAE02A
:10107C000E941822DF01E0915103F0915203EA170C
:10108C00FB0730F40E94F61B0E940B1C0E94AA1A4C
:10109C001333A0F0E0E0E0931703E12FF0E0F297B8
:1010AC000E9498210E941920A6EFB8E28CE99FE3D8
:1010BC000E94A3200E94E01F1E2F01C010E00E947E
:1010CC00DF1AEB83FC83AB2DE4E60E94B6210E2ED7
:1010DC00A0E0F099A1E0E1E00E94A2210E94201A78
:1010EC001E2E0E94101CA0914303B09144030E9439
:1010FC00C0210E94151C0E94281AE021E129E9F068
:10110C00E0912D03F0912E03ABE1B0E00E94E722B9
:10111C000E941D1C0E94791CE0910803A8E1B0E01C
:10112C000E94EF22A4E6B0E00E94A91F5F98A8EEEF
:10113C00B3E00E94A91F0C940019E0911103E093F5
:10114C00B300AA2D0E94D81C0E94721BE02131F022
:10115C00E894F2F827F8E0E0E09326030E94DD1C07
:10116C000E94721BE02171F0E0912603EF5FE09387
:10117C002603A0912603AA3029F4E0E0E09326038D
:10118C00E09319030E94DD1C0E94EA1C0E94721B52
:10119C00E02171F06894F2F8E0911903EF5FE093AD
:1011AC001903A0911903A33019F4E1E0E09319039A
:1011BC00E0911903E03029F4E0E0E093B400F798F3
:1011CC000FC0A0911903A13019F4E091120306C0CD
:1011DC00A0911903A23021F4F79AEFEFE093B40039
:1011EC000E9412190E944B190E2EA12F0E947E1BD9
:1011FC0001F1E0910403EF5FE0930403A091040379
:10120C00E5E00E94BB210E2EE4E10E94B621E02114
:10121C0041F0E0910403E170AFEFEA02F001E093DA
:10122C00B400A0910403A03118F0E0E0E0930403B3
:10123C0026C0A0E030FCA1E0E1E00E94A2210E2E2D
:10124C00A09119030E948A1BD1F0E0912503EF5F56
:10125C00E0932503A0912503A13019F4EFEFE0935F
:10126C00B400A0912503A33019F4E0E0E093B4009E
:10127C00A0912503A43019F4E0E0E0932503EAE003
:10128C00E81518F4E894F1F826F80E94F21CA0E096
:10129C0026FCA1E00E94F81CA0E0F1FCA1E00E9459
:1012AC00F81C0E94721BE02131F06894F1F82F5F5A
:1012BC00283009F420E00E94F21CA0911403EFEFF7
:1012CC000E94B621E02121F0E0911403EF5F03C0EE
:1012DC00E894F1F8E0E0E0931403A0911403A43136
:1012EC00A9F4AA81E0E00E94B1210E2E0E94721B8B
:1012FC00E02119F0EA81E150EA83233610F423E669
:10130C0005C020E00E941D1C0E94791C0E94F21C4A
:10131C00A0E0F1FCA1E00E94F81CAA81E4E60E9486
:10132C00AC210E94FD1C51F06894F1F8EA81EF5F4A
:10133C00EA83AA81A43611F4E0E0EA83EAE0E91535
:10134C0010F4E894F0F80E946C1B0E94771B0E229C
:10135C00AA81E0E00E94A7210E94FD1C51F0689434
:10136C00F0F8EA81E150EA83AA81AF3F11F4E3E699
:10137C00EA830E94CF1A0E94041DC1F00E940A1D2C
:10138C00A9F4A0912303A43119F4E7E0E09323031B
:10139C00E0E0E0932403E894F3F8A0912303A33056
:1013AC0028F0E0912303E150E0932303AA2DEAE017
:1013BC000E94B6210E2E0E94041DC1F00E940A1D2F
:1013CC00A9F4A0912303A43119F4E7E0E0932303DB
:1013DC00E0E0E0932403E894F2F8A0912303A33017
:1013EC0028F0E0912303E150E0932303AA2D0E94FF
:1013FC00D81CAD2DEAE00E94BB21E02131F0E0E0E9
:10140C00E0932403E4E1E0932303EAE0ED1510F408
:10141C00E894F3F80E94CF1A0E94D51A0E94A221D8
:10142C00E02109F495C16894F3F8AA81A13049F43C
:10143C00A0910B03A13028F4E0910B03EF5FE09334
:10144C000B03AA81A23049F4A0910C03A23328F417
:10145C00E0910C03EB5FE0930C03AA81A33049F4F9
:10146C00A0910D03A43628F4E0910D03EE5FE093F8
:10147C000D03AA81A43049F4A0910F03A83228F4DB
:10148C00E0910F03EF5FE0930F03AA81A53031F4D5
:10149C00AE89A43618F4EE89EF5FEE8BAA81A630E4
:1014AC0031F4AF89A43618F4EF89EF5FEF8BAA8182
:1014BC00A73031F4A88DA43618F4E88DEF5FE88FCF
:1014CC00AA81A83049F4A0911003AF3F28F4E09111
:1014DC001003EF5FE0931003AA81AD3069F4A09183
:1014EC002F03B0913003A433E8E0BE0728F40E9428
:1014FC009E1A31960E946E1AAA81AE3031F4AA89D6
:10150C00A43618F4EA89EB5FEA8BAA81AF3031F488
:10151C00AB89A43618F4EB89EB5FEB8BAA81A03175
:10152C0031F4AC89A43618F4EC89EB5FEC8BAA810E
:10153C00A13131F4AE85A83C18F4EE85EB5FEE8753
:10154C00AA81A23131F4AF85A83C18F4EF85EB5F8A
:10155C00EF87AA81A33131F4A889A83C18F4E88953
:10156C00EB5FE88BAA81A43169F4A0914103B0919F
:10157C004203A835E2E0BE0728F40E94101C7E96B8
:10158C000E94841AAA81A53159F4AD81BE81A33A77
:10159C00E1E0BE0728F4ED81FE813196ED83FE83F8
:1015AC00AA81A63149F4A0911A03A13028F4E09144
:1015BC001A03EF5FE0931A03AA81A73149F4A091B3
:1015CC001C03A23328F4E0911C03EF5FE0931C038F
:1015DC00AA81A83149F4A0911B03A13028F4E09111
:1015EC001B03EF5FE0931B03AA81A93119F43F3071
:1015FC0008F43F5FAA81AA3159F40E94151DAC3B37
:10160C00E2E0BE0728F40E941A1D31960E947A1A55
:10161C00AA81AB3159F40E947A19A73EE3E0BE07C8
:10162C0028F40E941F1D31960E947F1AAA81AC31AA
:10163C0061F4A0E023FCA1E0A13038F4E0E023FC4D
:10164C00E1E0EF5F0E941A2323F8AA81AD3169F41F
:10165C000E944619AE3DE3E0BE0738F40E942719FC
:10166C003A96E0933703F0933803AA81AE3169F4CC
:10167C000E945019A835E2E0BE0738F40E943319D5
:10168C003A96E0934503F0934603AA81AF3149F4AF
:10169C00A0910803AA3028F4E0910803EF5FE093CF
:1016AC000803AA81AC3549F4A0910703AA3F28F49A
:1016BC00E0910703E65FE0930703AA81AD3531F4AF
:1016CC00AB8DA73018F4EB8DEF5FEB8FAA81AE35A5
:1016DC0049F4A985BA851A9728F4E985FA853196D3
:1016EC00E987FA87AA81AF3531F4AA8DAA3018F4AC
:1016FC00EA8DEF5FEA8FAA81A03631F4A98DAA306A
:10170C0018F4E98DEF5FE98FAA81A13649F4A09115
:10171C001503AC3328F4E0911503EF5FE093150348
:10172C00AA81A23649F4A0911203AA3F28F4E091B1
:10173C001203E65FE0931203AA81A33649F4A09149
:10174C001103AA3F28F4E0911103E65FE093110323
:10175C00EAE0EA1510F4E894F2F8AA2DEAE00E9407
:10176C00B6210E2E0E94EA1C0E94041D09F492C19F
:10177C006894F2F8AA81A13049F4A0910B03A1302E
:10178C0028F0E0910B03E150E0930B03AA81A23007
:10179C0049F4A0910C03AB3028F0E0910C03E55018
:1017AC00E0930C03AA81A33049F4A0910D03AD334F
:1017BC0028F0E0910D03E250E0930D03AA81A430D0
:1017CC0049F4A0910F03A53128F0E0910F03E150EB
:1017DC00E0930F03AA81A53031F4AE89A13018F043
:1017EC00EE89E150EE8BAA81A63031F4AF89A1309D
:1017FC0018F0EF89E150EF8BAA81A73031F4A88D56
:10180C00A13018F0E88DE150E88FAA81A83049F496
:10181C00A0911003A13028F0E0911003E150E09367
:10182C001003AA81AD3069F4A0912F03B09130035D
:10183C00AD36E7E0BE0728F00E949E1A31970E9451
:10184C006E1AAA81AE3031F4AA89A63018F0EA8952
:10185C00E550EA8BAA81AF3031F4AB89A63018F091
:10186C00EB89E550EB8BAA81A03131F4AC89A63021
:10187C0018F0EC89E550EC8BAA81A13131F4AE85DE
:10188C00A13018F0EE85E550EE87AA81A23131F433
:10189C00AF85A13018F0EF85E550EF87AA81A33111
:1018AC0031F4A889A13018F0E889E550E88BAA81B9
:1018BC00A43161F4A0914103B09142030E9406232C
:1018CC0028F40E94101C7E970E94841AAA81A531CC
:1018DC0059F4AD81BE81A332E1E0BE0728F0ED8161
:1018EC00FE813197ED83FE83AA81A63149F4A09144
:1018FC001A03A13028F0E0911A03E150E0931A0387
:10190C00AA81A73149F4A0911C03A23028F0E091E0
:10191C001C03E150E0931C03AA81A83149F4A09167
:10192C001B03A13028F0E0911B03E150E0931B0353
:10193C00AA81A93119F4323008F03150AA81AA31A8
:10194C0059F40E94151DA935E2E0BE0728F00E944B
:10195C001A1D31970E947A1AAA81AB3149F40E9460
:10196C007A191B9728F00E941F1D31970E947F1A2D
:10197C00AA81AC3179F4A0E023FCA1E0A13050F0B5
:10198C00A0E023FCA1E0E1E00E94C722EA1B0E9438
:10199C001A2323F8AA81AD3161F40E9446190E94E2
:1019AC00062338F40E9427193197E0933703F093FC
:1019BC003803AA81AE3161F40E9450190E940623AB
:1019CC0038F40E9433193197E0934503F0934603A2
:1019DC00AA81AF3149F4A0910803A23028F0E0911C
:1019EC000803E150E0930803AA81AC3539F4A091C7
:1019FC000703A13018F0E0E0E0930703AA81AD35AE
:101A0C0031F4AB8DA13018F0EB8DE150EB8FAA8146
:101A1C00AE3551F4A985BA850E94062328F4E985D0
:101A2C00FA853197E987FA87AA81AF3531F4AA8D07
:101A3C00A13018F0EA8DE150EA8FAA81A03631F47A
:101A4C00A98DA13018F0E98DE150E98FAA81A1365A
:101A5C0049F4A0911503A13028F0E0911503E15051
:101A6C00E0931503AA81A23649F4A0911203AB307E
:101A7C0028F0E0911203EA50E0931203AA81A336F6
:101A8C0049F4A0911103A13028F0E0911103EA5020
:101A9C00E093110323FC26C0E0912103A3EAB3E0F9
:101AAC00FF27662777270E9419200E94B422A09155
:101ABC00A303B091A4038091A5039091A6030E9467
:101ACC000A233CF40E94241D0E942D1D0E94341DEB
:101ADC0009C0E0E0E0939303E0939403E093950353
:101AEC00E093960323FE0CC0AC85B0E00E940B1C67
:101AFC00A3EAB3E00E94731A0E94241D0E94341DB5
:101B0C000E94241DAFE1B3E00E94E01FEC93F09122
:101B1C004703E0E0DF01E0912203F0E0EA0FFB1F56
:101B2C00A3E7B3E00E942C190E943D1DA0E0B0E099
:101B3C0080E192E40E94F1207F936F93FF93EF93E7
:101B4C000E94151D0E94461DAF91BF918F919F91D0
:101B5C000E94EF1BE0937303F0937403609375037F
:101B6C00709376030E944B1DE0E0F0E060E87FE3A9
:101B7C000E945C210E2E0E944B1DE0E0F0E068E418
:101B8C0072E40E945621E021F9F00E943D1D0E9452
:101B9C002D1DA3E6B3E00E94E21F0E94B4220E9416
:101BAC003D1DE0937703F093780360937903709372
:101BBC007A030E944B1D0E9441190E94A320A1E3AD
:101BCC00B3E00E945E1915C0E0E0E0936303E0937C
:101BDC006403E0936503E0936603E0937703E0937B
:101BEC007803E0937903E0937A03E0933103E09375
:101BFC003203A0919703B09198038091990390912F
:101C0C009A030E940D1A0E945C21EF930E94541DAE
:101C1C000E945C21AF91EA23C9F10E947119E0E0A6
:101C2C00F0E068EC72E40E94F1200E947A19882797
:101C3C0099270E94BB220E9490190E94561DA091C8
:101C4C006F03B09170038091710390917203E0E087
:101C5C00F0E064E172E40E94A320DF01CB010E945A
:101C6C00BC190E94F120A0E0B0E080E291E40E9457
:101C7C00A3200E94561DE0916F03F09170036091B8
:101C8C00710370917203DE010E9495190E946C1B06
:101C9C00A0911303EDEF0E94B6210E220E94721B3D
:101CAC00E02129F0E0911303EF5FE0931303A92DDA
:101CBC000E94D81CA0911303EFEF0E94B6210E22B4
:101CCC000E94721BE02129F0E894F0F8E0E0E09328
:101CDC001303A0911303EEE10E94A2210E2E0E9489
:101CEC00721BE02119F0E1E0E0931603E09115037B
:101CFC00E03019F4E0E0E09316030E94171A0E94FA
:101D0C000D1A0E94E8210E94151CA09116030E9436
:101D1C007E1B19F0E1E0E0931603A0911603AC339F
:101D2C0009F41FEFA0910703A13028F0E0910703FD
:101D3C00F0E00E94AA1A4420C9F4E02FF0E0349697
:101D4C000E941219AE0FBF1FE12F0E945F1DA4E06D
:101D5C000E940319A02F0E94691DA09127030E94C5
:101D6C000319A12F0E9403190E946E1DE1E0E415D6
:101D7C0009F057C04424A0910D030E94771DE093F5
:101D8C000E03F0E0BC96DF01E0910A03F0E0AE0F29
:101D9C00BF1FE0910B03F0E0AE0FBF1FE0910C03EF
:101DAC00F0E0AE0FBF1FE0910F03F0E0AE0FBF1FCE
:101DBC00EE89F0E0AE0FBF1FEF89F0E0AE0FBF1F52
:101DCC00E88DF0E0AE0FBF1FE09110030E945F1D85
:101DDC00ACE20E940319A0910A030E940319A0917E
:101DEC000B030E940319A0910C030E940319A091EC
:101DFC000E030E940319A0910F030E940319AE89D0
:101E0C000E940319AF890E940319A88D0E9403191F
:101E1C00A09110030E94691DA0E00E94691D0E9400
:101E2C006E1D233608F059C3A0E0F799A1E0EA2F04
:101E3C00E295E07F0E2EA0E0F399A1E0EA2FEE0FE1
:101E4C00EE0F0E0EA0E0F499A1E0EA2FEE0FA02DFC
:101E5C00AE0FE0E0F599E1E0EA0FEC8FEAE0E9ABD8
:101E6C00EAABEBABECABEDABEEABEFAB0E947D1D9D
:101E7C00EAE0EBAFECAFEDAFEEAFEFAF0E94821D3F
:101E8C00AA34E1E0BE07E0E08E07E0E09E071CF418
:101E9C00E1E0E09302030E94821DE9E4F1E060E0DE
:101EAC0070E00E948B1DEEE5F1E060E070E00E94B6
:101EBC00E021E02119F0E3E0E09302030E94821D8F
:101ECC00EDE5F1E060E070E00E948B1DE8E6F1E0EA
:101EDC0060E070E00E94E021E02119F0E7E0E0937F
:101EEC0002030E94821DE7E6F1E060E070E00E94D0
:101EFC008B1DECE7F1E060E070E00E94E021E02156
:101F0C0019F0EFE0E09302030E94821DAC37E1E090
:101F1C00BE07E0E08E07E0E09E071CF0EFE1E093E7
:101F2C0002030E94171A0E948F1D2CF00E94971D0D
:101F3C000E949D1DEBAB0E94971D0E947F22ECAB73
:101F4C00A0911F03AA3030F0B0E00E940B1C0E943D
:101F5C00A81DE9AB0E94AE1DEAAB0E94821D0E9437
:101F6C00B61D0E949D1DEDAB0E94BB1D0E949D1DC8
:101F7C00EEAB0E94BB1D0E947F22EFAB203099F587
:101F8C000E94C11DE7550E94C71D0E94D11DA43699
:101F9C00E0E0BE0720F00E94D11D0E94D61D0E94D9
:101FAC00D11D0E94461D0E94E11DEEAF0E94D11D65
:101FBC000E94E71DEFAFA0910103AA3010F0E2E000
:101FCC00E8AFA09101030E94EC1DE9AFA0910003C2
:101FDC00B0E00E940B1C0E94A81DEAAFA091000368
:101FEC000E94EC1DEBAF213009F05CC00E94F21D89
:101FFC00E75B0E94C71D0E94041AA03AE6E8BE07E0
:10200C00E1E08E07E0E09E0748F00E94041AE0EA47
:10201C00F6E861E070E00E94F51DEAAF0E94041A38
:10202C00A031E7E2BE07E0E08E07E0E09E0748F053
:10203C000E94041AE0E1F7E260E070E00E94F51DF6
:10204C00EBAF0E94041AA83EE3E0BE07E0E08E0767
:10205C00E0E09E0738F00E94041A0E94611B0E9467
:10206C00F51DECAF0E94041AA436E0E0BE07E0E0D8
:10207C008E07E0E09E0738F00E94041A0E94B61DFD
:10208C000E94F51DEDAF0E94041A0E948F1D28F0CE
:10209C000E94001E0E94F51DEEAF0E94001E0E94C1
:1020AC007B22EFAF223009F06AC00E94F21DE75F7D
:1020BC000E94C71DE7E7E9AFE4E7EAAFA091580338
:1020CC00AA2352F4E0915703F09158030E946C211B
:1020DC00E0935703F09358030E94541D0E949019EB
:1020EC00772312F4E0E4EEAF0E94541D0E94901985
:1020FC000E94061E10F4E0E4EDAF0E94541D0E94F5
:10210C0090190E940F1E10F4E0E4ECAF0E94541DD5
:10211C000E9490190E94181E10F4E0E4EBAF0E948C
:10212C00211EA031E7E2BE072CF00E94211E0E9466
:10213C00261EEBAF0E94211EA83EE3E0BE072CF04A
:10214C000E94211E0E942B1EECAF0E94211EA43661
:10215C00E0E0BE072CF00E94211E0E94301EEDAF65
:10216C000E94211E1A973CF00E94211E0E940B1CFB
:10217C000E94A81DEEAF0E94211E0E94351E233026
:10218C0009F062C00E94F21DE7570E94C71DEEE3E2
:10219C00E9AFE4E7EAAFA0915A03AA2352F4E09125
:1021AC005903F0915A030E946C21E0935903F09368
:1021BC005A030E943B1E772312F4E0E4EEAF0E9418
:1021CC003B1E0E94061E10F4E0E4EDAF0E943B1E85
:1021DC000E940F1E10F4E0E4ECAF0E943B1E0E9424
:1021EC00181E10F4E0E4EBAF0E943E1EA031E7E2B3
:1021FC00BE072CF00E943E1E0E94261EEBAF0E94D2
:10220C003E1EA83EE3E0BE072CF00E943E1E0E943C
:10221C002B1EECAF0E943E1EA436E0E0BE072CF055
:10222C000E943E1E0E94301EEDAF0E943E1E1A9769
:10223C003CF00E943E1E0E940B1C0E94A81DEEAF9B
:10224C000E943E1E0E94351E243001F50E94F21D94
:10225C00E7570E94C71DEEE3E9AFE4E7EAAFE0E51C
:10226C00EBAFA0911E03A43620F0B0E00E94301E0C
:10227C00EDAFA0911E03B0E00E940B1C0E94A81DA4
:10228C00EEAFA0911E030E94EC1DEFAF253041F57F
:10229C000E94F21DE7570E94C71DE0E0E9AFE5E0A0
:1022AC00EAAFE8E7EBAFA881B981A83EE3E0BE074F
:1022BC001CF00E942B1EECAFA881B981A436E0E083
:1022CC00BE071CF00E94301EEDAFA881B9810E94A0
:1022DC000B1C0E94A81DEEAFA881B9810E94351E6F
:1022EC00263009F04CC00E94F21DE75F0E94C71D0A
:1022FC00113030F1ECE0E9AFA12F0E94771DE436EC
:10230C00A0E0FA074CF0A12FB0E0E8ECF0E00E945E
:10231C003B220E94A81DEAAFA12F0E94771D3A977D
:10232C004CF0A12FB0E0E4E1F0E00E943B220E94CF
:10233C00A81DEBAFA12F0E94771D0E94A81D1EC0E7
:10234C00EBE0E9AF0E94431EE436A0E0FA0738F058
:10235C00AB81BC81E8ECF0E00E94481EEAAF0E9421
:10236C00431E3A9738F0AB81BC81E4E1F0E00E9467
:10237C00481EEBAF0E94431E0E94E11DECAF2730BC
:10238C0009F074C0A0915303B0915403A135EBEF45
:10239C00BE0734F4E1E5FBEFE0935303F0935403F1
:1023AC00A0915303B0915403A03BE4E0BE0734F07A
:1023BC00EFEAF4E0E0935303F0935403A091540339
:1023CC00AA234AF4E0E4ECAFE0915303F0915403F8
:1023DC000E946C2104C0E0915303F0915403E093EC
:1023EC005503F0935603A0915503B0915603ECE3BB
:1023FC00F0E00E943B22E0933B03F0933C030E94ED
:10240C004B1EECE30E941822A0915503B091560389
:10241C00AE1BBF0BA0933D03B0933E030E94C11DA6
:10242C00E75D0E94C71D24FE1BC00E944B1E1A971D
:10243C0010F0E2E0E8AF0E944B1E0E94E71DE9AFEE
:10244C00A0913D03B0913E030E94461D0E94E11DE8
:10245C00EAAFA0913D03B0913E030E94E71DEBAFA4
:10246C00E3E7EDAFE8E3EEAFE4E5EFAF0E94501E1B
:10247C00AE2FE09120030E94561EEA0F0E945C1EB4
:10248C000E94651EED8FAB85A130E8F00E947D1D8A
:10249C00E9E7EBAFE0E5ECAFEDAFAB85B0E00E9468
:1024AC000B1C0E94A81DEEAFAB850E94EC1DEFAF7C
:1024BC000E94501E0E945C1EE00DED8F0E94C11DFB
:1024CC00E75F0E94C71DF29B08C00E94501E0E942D
:1024DC005C1E0E94651EEF5FED8F233609F09DC3D5
:1024EC0051E0503130F40E946E1EEAE0EC935F5FD5
:1024FC00F8CFAA81EBE50E94751EEAE50E94A221A5
:10250C00E02911F0EFE1EA83AA81A03211F4ECE5A5
:10251C00EA83EA81E03029F4E0910A03F0E0EF83EA
:10252C00F887AA81A13029F4E0910B03F0E0EF8346
:10253C00F887AA81A23029F4E0910C03F0E0EF8334
:10254C00F887AA81A33029F4E0910D03F0E0EF8322
:10255C00F887AA81A43029F4E0910F03F0E0EF830F
:10256C00F887AA81A53021F4EE89F0E0EF83F88793
:10257C00AA81A63021F4EF89F0E0EF83F887AA81D5
:10258C00A73021F4E88DF0E0EF83F887AA81A8301A
:10259C0029F4E0911003F0E0EF83F887AA81A930C9
:1025AC0019F4E0E0EF83E887AA81AA3019F4E0E09F
:1025BC00EF83E887AA81AB3019F4E0E0EF83E8877A
:1025CC00AA81AC3021F4E4E2F0E0EF83F887AA8131
:1025DC00AD3021F40E949E1AEF83F887AA81AE30A9
:1025EC0021F4EA89F0E0EF83F887AA81AF3021F477
:1025FC00EB89F0E0EF83F887AA81A03121F4EC8914
:10260C00F0E0EF83F887AA81A13121F4EE85F0E0A8
:10261C00EF83F887AA81A23121F4EF85F0E0EF83F4
:10262C00F887AA81A33121F4E889F0E0EF83F887D9
:10263C00AA81A43121F40E94101CEF83F887AA818F
:10264C00A53121F4ED81FE81EF83F887AA81A631B3
:10265C0029F4E0911A03F0E0EF83F887AA81A731FF
:10266C0029F4E0911C03F0E0EF83F887AA81A831EC
:10267C0029F4E0911B03F0E0EF83F887AA81A931DC
:10268C0021F4E32FF0E0EF83F887AA81AA3121F43B
:10269C000E941A1DEF83F887AA81AB3121F40E94A6
:1026AC001F1DEF83F887AA81AC3131F4E0E023FCE5
:1026BC00E1E0F0E0EF83F887AA81AD3121F40E94CC
:1026CC002719EF83F887AA81AE3121F40E943319C0
:1026DC00EF83F887AA81AF3129F4E0910803F0E089
:1026EC00EF83F887AA81AC3529F4E0910703F0E079
:1026FC00EF83F887AA81AD3521F4EB8DF0E0EF8301
:10270C00F887AA81AE3521F4E985FA85EF83F8873D
:10271C00AA81AF3521F4EA8DF0E0EF83F887AA8126
:10272C00A03621F4E98DF0E0EF83F887AA81A13679
:10273C0029F4E0911503F0E0EF83F887AA81A23623
:10274C0029F4E0911203F0E0EF83F887AA81A33615
:10275C0029F4E0911103F0E0EF83F887AA81E0E01F
:10276C000E94751EE3E00E947A1EE1E10E947A1E2F
:10277C00E2E10E947A1EE3E10E947A1EE5E10E94EA
:10278C007A1EEBE10E947A1EEDE10E94A221E02963
:10279C0011F0F69A01C0F698A0E0F699A1E0EA2FA4
:1027AC00E795E0E0E795EE8FE0E0ED8FEC8FE093BE
:1027BC000203AA81B0E0A7FDBFEF0E940B1C0E9490
:1027CC00A81DEBABAA81B0E0A7FDBFEFEAE0F0E0FB
:1027DC000E946D22ECABAF81B885A031E7E2BE0759
:1027EC0028F0E0E1F7E20E94481EEBAFAF81B8851C
:1027FC00A83EE3E0BE0728F0E8EEF3E00E94481E96
:10280C00ECAFAF81B885A436E0E0BE0710F00E94B3
:10281C00D61DAF81B8851A9728F00E947F1E0E94A2
:10282C00E11DEEAFAF81B8850E94E71DEFAFEA81E5
:10283C00E03061F4EDE6EDABE9E7EEABE8E7EFABEA
:10284C00EDE6EAAFE4E5EBAFE0E5ECAFAA81E1E160
:10285C000E94751EE2E10E947A1EE3E10E947A1E3C
:10286C00E5E10E947A1EEDE10E94A221E02929F007
:10287C000E947F1E0E94E11DEEAFE7EAE0937A0012
:10288C00A7E00E94891A0E94AA1AE7E2E0937A0054
:10289C00AA810E94C51AAA81EEE00E947A1EE1E18B
:1028AC000E94A221E02911F0E1E06E2EAA810E9483
:1028BC00CA1AAA81EFE00E947A1EE2E10E94A221CC
:1028CC00E02911F0E2E06E2EAA81E7E00E94751E6D
:1028DC00E0E10E947A1E0E94821E11F0E3E06E2E4F
:1028EC000E941219D39708F457C00E94DF1A0E9455
:1028FC00E41AE62D0E94EB1A20F0E8ECF0E00E94BE
:10290C00AA1AE62D0E94FB1A0E94871EAC91A130D8
:10291C0008F441C00E948E1E0E941B1B0E941523AE
:10292C004CF40E94871E0E94971E0E9462210E94F6
:10293C00A21E23C00E94AB1E0E943D1BEF930E945F
:10294C00AB1E0E94461BAF91EA2379F00E94871EB2
:10295C000E94971E0E946721A0935F03B0936003AF
:10296C00809361039093620308C00E94AB1E0E9487
:10297C004F1B1CF00E94AD1E0EC0A0915F03B091C6
:10298C00600380916103909162030E94611B0E941D
:10299C0065220E94AA1A04C00E94661B0E94AD1EEA
:1029AC00AA81AD3061F40E94B51E0E94B61D0E9432
:1029BC009D1D0E94BE1E0E94C51EE0E2EC8FAA81E6
:1029CC00A53161F40E94B51E0E94B61D0E949D1D8A
:1029DC000E94BE1E0E94C51EE0E6EC8FAA810E94DA
:1029EC00C51AAA81EEE00E947A1EE1E10E94A221A2
:1029FC00E029A9F00E94CF1EE4E00E94D31E18F03B
:102A0C000E94D91EEDAB0E9412191A9728F00E9451
:102A1C00DD1E0E94E11DEEAB0E94DF1EEFABAA8112
:102A2C000E94CA1AAA81EFE00E947A1EE2E10E947B
:102A3C00A221E029A9F00E94CF1EE2E00E94D31E41
:102A4C0018F00E94D91EEDAB0E9412191A9728F0AB
:102A5C000E94DD1E0E94E11DEEAB0E94DF1EEFAB5B
:102A6C00AA81E7E00E94751EE0E10E947A1E0E9496
:102A7C00821EA9F00E94CF1EE1E00E94D31E18F026
:102A8C000E94D91EEDAB0E9412191A9728F00E94D1
:102A9C00DD1E0E94E11DEEAB0E94DF1EEFABAA8192
:102AAC00A63121F40E94E11EEBE0ECAFAA81A73124
:102ABC0021F40E94E11EE0E4ECAFAA81A83121F4DC
:102ACC000E94E11EECE0ECAFAA81A93169F4A0915F
:102ADC001F03B0E00E940B1C0E94A81DEDAB0E94CE
:102AEC00AE1DEEABE7E7EFABAA81AA3199F40E94D9
:102AFC00E81EE4E6F0E00E94481EEDAB0E94E81EE2
:102B0C000E94461D0E94E11DEEAB0E94E81E0E9431
:102B1C00E71DEFABAA81AB3159F4ECE7E9AFE7E77E
:102B2C00EAAFE8E7EBAF0E947F1E0E94E11DEEAF1B
:102B3C00AA81EDE10E94751EEEE10E94A221E0291E
:102B4C00D9F0E3E7E9AFE8E3EAAFAA81AD3111F4DC
:102B5C00EEE501C0E8E7EBAF0E94ED1E1A9738F0E6
:102B6C000E94ED1E0E94461D0E94E11DEEAB0E94CC
:102B7C00ED1E0E94E71DEFABAA81E1E10E94751EDC
:102B8C00E2E10E947A1E0E94821E11F0E8E7EAAF91
:102B9C00AA81AD3541F5E7E7ECAFEEE5EDAFE9E342
:102BAC00EEAFEB8DEFAFE7EAE0937A00AB8D0E94CE
:102BBC00891A7E2EE7E2E0937A00E3E6E71528F423
:102BCC00A72DB0E00E94301EEDABE9E0E71538F41C
:102BDC00A72DB0E00E940B1C0E94A81DEEABA72DE8
:102BEC000E94EC1DEFABAA81AE3521F4EEE5E9AF06
:102BFC00E1E0EAAFAA81AF3521F4EEE5E9AFE2E01E
:102C0C00EAAFAA81A03621F4EEE5E9AFE3E0EAAF42
:102C1C00AA81A23611F4E0E1EC8F51E0503108F0BA
:102C2C0077C00E946E1EEC91E03021F40E946E1E63
:102C3C00EFE3EC930E946E1EAC91A63021F40E943F
:102C4C006E1EEDE7EC930E946E1EAC91A13021F448
:102C5C000E946E1EE6E0EC930E946E1EAC91A230B8
:102C6C0021F40E946E1EEBE5EC930E946E1EAC915B
:102C7C00A33021F40E946E1EEFE4EC930E946E1EB2
:102C8C00AC91A43021F40E946E1EE6E6EC930E94F7
:102C9C006E1EAC91A53021F40E946E1EEDE6EC93F5
:102CAC000E946E1EAC91A73021F40E946E1EE7E0CC
:102CBC00EC930E946E1EAC91A83021F40E946E1E03
:102CCC00EFE7EC930E946E1EAC91A93021F40E94A8
:102CDC006E1EEFE6EC930E946E1EAC91AA3021F4AE
:102CEC000E946E1EE0E0EC930E946E1EAC91AB3025
:102CFC0021F40E946E1EE1E0EC930E946E1EAC91DA
:102D0C00AC3021F40E946E1EE8E0EC935F5F86CF3E
:102D1C00E0910203E695E6950E94F21EEDA90E9451
:102D2C00F81EEDA90E94031FEDA90E940E1FEDA92C
:102D3C000E94151FEDA90E941C1FEDA90E94231FC4
:102D4C00EDA90E942A1FE8A3E0910203E695E695FF
:102D5C00E6950E94F21EEEA90E94F81EEEA90E94B2
:102D6C00031FEEA90E940E1FEFA90E94151FEFA9C9
:102D7C000E941C1FEFA90E94231FEFA90E942A1F6B
:102D8C00E9A3E0910203E6950E94F21EEFA90E94CE
:102D9C00F81EEFA90E94031FEFA90E940E1FEEA9B7
:102DAC000E94151FEEA90E941C1FEEA90E94231F52
:102DBC00EEA90E942A1FEAA3E8AD0E94F21EE9AD1B
:102DCC000E94F81EE9AD0E94031FE9AD0E940E1F80
:102DDC00EE8D0E94151FEE8D0E941C1FEE8D0E9421
:102DEC00231FE0910203E170EA2BEBA3EDAD0E94EF
:102DFC00F21EEDAD0E94301FEDAD0E94391FEDADFE
:102E0C000E94421F0E944C1FEDAD0E94501FEDAD61
:102E1C000E94591FEDADE295E170EA2BECA3ECADED
:102E2C000E94F21EECAD0E94301FECAD0E94391FC7
:102E3C00ECAD0E94421FE2950E94151FEEAD0E9460
:102E4C00501FEEAD0E94591FEEADE295E170EA2BDA
:102E5C00EDA3EE8D0E94621FECAD0E94F81EECAD4E
:102E6C000E94031FECAD0E940E1FEBAD0E94151FBC
:102E7C00EBAD0E941C1FEBAD0E94231FEBAD0E941B
:102E8C002A1FEEA3EEAD0E94F21EEEAD0E94301F83
:102E9C00EEAD0E94391FEEAD0E94421F0E94661FCC
:102EAC000E94151FEBAD0E94501FEBAD0E94591FE5
:102EBC00EBADE295E170EA2BEFA3EAAD0E94F21EB6
:102ECC00EAAD0E94301FEAAD0E94391FEAAD0E94A4
:102EDC00421FEE1FE0E0EE1F0E94151FEFAD0E9497
:102EEC00501FEFAD0E94591FEFADE295E170EA2B38
:102EFC00E8A7ED8DE2950E94F21EEAAD0E94F81E45
:102F0C00EAAD0E94031FEAAD0E940E1FE9AD0E94BC
:102F1C00151FE9AD0E941C1FE9AD0E94231FE9ADEE
:102F2C000E942A1FE9A7EFAD0E94F21EEFAD0E948E
:102F3C00301FEFAD0E94391FEFADE695E695E69593
:102F4C000E946B1FE9A9EE1FE0E0EE1F0E94151F07
:102F5C00E9A9E295E170EE0FEE0FEA2BAE2FE9A98D
:102F6C000E94591FE9A9E295EF70E695E170EA2BF2
:102F7C00EAA7E9A9E695E695E6950E94F21EE9A96D
:102F8C00E695E6950E94711FE9A90E94791FE9A9AF
:102F9C000E946B1FED8D0E944C1FED8D0E94561EE2
:102FAC00EA2BAE2FED8D0E94811FED8DE695E17021
:102FBC00EA2BEBA7ED8D0E94621FEAA9E2950E9415
:102FCC00711FEAA90E94031FEAA90E94861FEAA9A1
:102FDC000E944C1FEAA90E94561EEA2BAE2FEAA9AA
:102FEC00E6950E94811FEAA9E170EA2BECA7ED8D12
:102FFC000E94661F0E94F21EEC8D0E94711FEC8DC8
:10300C000E94791FEC8DE695E6950E946B1FE0916E
:10301C000203E2950E94151FED8DEE1FE0E0EE1FFE
:10302C00E170EE0FEE0FEA2BAE2FEC8DE695E695E8
:10303C00E6950E94811FEC8DE295E170EA2BEDA7DD
:10304C00EC8D0E94621FEBA9E2950E94711FEBA907
:10305C000E94031FEBA90E94861FECA90E944C1F23
:10306C00ECA90E94561EEA2BAE2FECA9E6950E9405
:10307C00811FECA9E170EA2BEEA7EC8D0E94661F74
:10308C000E94F21EECA9E2950E94711FECA90E940D
:10309C00031FECA90E94861FEBA90E944C1FEBA9F1
:1030AC000E94561EEA2BAE2FEBA9E6950E94811FBB
:1030BC00EBA9E170EA2BEFA70E948A1F5D3078F430
:1030CC000E94901FA2E5B8E00E948021E17011F4EB
:1030DC005D9801C05D9A0E94971F5F5FEFCF0E94C1
:1030EC009F1F5D3078F40E94901FA0E3B8E00E940F
:1030FC008021E17011F45D9801C05D9A0E94971FC8
:10310C005F5FEFCF0E949F1F5D3078F40E94901F8D
:10311C00A2E0B8E00E948021E17011F45D9801C03A
:10312C005D9A0E94971F5F5FEFCF0E949F1F5D30DB
:10313C0078F40E94901FA6E0B8E00E948021E17014
:10314C0011F45D9801C05D9A0E94971F5F5FEFCFED
:10315C000E949F1F5A3098F45E9885E28A95F1F789
:10316C00E9E0E51BA0E4B1E00E948021E17011F4DC
:10317C005D9801C05D9A0E94971F5F5FEBCF41E0A5
:10318C004131E8F451E05930C0F45E9885E28A95FB
:10319C00F1F7E42FF0E0DE015F96AE0FBF1FAC91AC
:1031AC00E8E0E51B0E947821E17011F45D9801C004
:1031BC005D9A0E94971F5F5FE6CF4F5FE1CF5D9AEC
:1031CC0085E28A95F1F7289A8DEC9AE00197F1F750
:1031DC00AB2DE4E60E94BB210E2EA0E0F099A1E0FD
:1031EC000E948A1B29F0A4E6B0E00E94A91FF09A65
:1031FC000C94C504EF962196FFCFAA93E091C000E2
:10320C00E072E1F3E881E093C60021960895A09165
:10321C002B03B0912C030895A0912703B0912803A0
:10322C000895A0917703B0917803809179039091E0
:10323C007A030895E0E0F0E061EE75E40E94F1207D
:10324C000895E0913703F0913803089566277727A6
:10325C000E9419200E94B4220895E0914503F09138
:10326C0046030895A0917F03B09180038091810360
:10327C00909182030895E0E0F0E060E271E408953B
:10328C00A0913703B09138030895E0E0F0E00E947C
:10329C00D2210895A0914503B09146030895E09181
:1032AC00A703F091A8036091A9037091AA03089554
:1032BC000E94E01FED93FC930895A0919303B091AD
:1032CC009403809195039091960308950E94A320F6
:1032DC00DF01CB01AFCFA0918F03B0919003809110
:1032EC009103909192030895A0913903B0913A0300
:1032FC000895E4E60E941822DF01E0918F03F0911B
:10330C0090036091910370919203882799270E94F2
:10331C00BB2208950E94BE220E944C2008950E9458
:10332C00E21FED93FC930895E0916703F09168031D
:10333C006091690370916A0308950E941822DF015D
:10334C00E091AF03F091B0036091B1037091B203BF
:10335C00882799270E94BB22DDCFE0919B03F09137
:10336C009C0360919D0370919E030895E0919703D7
:10337C00F09198036091990370919A030895A0912C
:10338C007B03B0917C0380917D0390917E03089523
:10339C00E0937B03F0937C0360937D0370937E0337
:1033AC000895A0918303B09184038091850390913B
:1033BC0086030895E0917B03F0917C0360917D037B
:1033CC0070917E030895A0918B03B0918C03809132
:1033DC008D0390918E030895E0914903F0914A0377
:1033EC0060914B0370914C030895E0934903F09363
:1033FC004A0360934B0370934C030895A0914903C7
:10340C00B0914A0380914B0390914C030895E0E0F6
:10341C00F0E060E070E00895E0E00E94BB210E2E29
:10342C000895A0916303B09164038091650390911A
:10343C00660308950E22A0911603ECE30E94B621B8
:10344C00E0210895A0914103B09142031ECFA4E165
:10345C00B0E00E94A91FE7EAE0937A000895A4E087
:10346C000E942803EF2FF0E09E2EE7E2E0937A0013
:10347C00E7EAE0937A000895A3E00E942803EF2F77
:10348C00F0E08E2EE7E2E0937A00E7EAE0937A0030
:10349C000895A1E00E942803EF2FF0E0AE2EE7E2A2
:1034AC00E0937A000895EBE0E093B803E8EBE09347
:1034BC00B9030895E8ECF0E0E0934F03F093500368
:1034CC000895E0EDF7E0E0935103F0935203089573
:1034DC00E0932F03F093300308950E9498210E94EB
:1034EC0019200E94B4220895E0933503F09336031B
:1034FC000895E0933903F0933A030895E093410360
:10350C00F093420308950E942803EF2FF0E00895F2
:10351C000E9428030E948D210E9489210895E09326
:10352C006703F09368036093690370936A030895CB
:10353C00E0912F03F09130030895E7E2E0937A00D5
:10354C00E7EAE0937A000895E0932703F0932803C9
:10355C00089562DEEAEFF0E008955EDEEEE1F0E061
:10356C000E94CC2108950E2EA52DE1E00E94BB21D6
:10357C000E22AB85E5E00E94B621E0210895E5E03E
:10358C000E94A2210E2E0895E6E00E94A2210E2E8A
:10359C000895AD2DEAE00E94B6210E2E0895A0E00C
:1035AC00F3FCA1E0E0E00E94A2210E22A22FE3E6B0
:1035BC000895E0912703F09128030895F297ADE761
:1035CC00B0E00E94F0210F010895F0E0DE01519669
:1035DC00AE0FBF1FEC91F0E0D0010E942822B4DFA7
:1035EC001BDEA93CE0E0BE070895F0E0DE01559635
:1035FC00AE0FBF1FEC91F0E00FDE0E94F021DF0157
:10360C00E4E6F0E00E9428229FCFE02FF0E0DE01FC
:10361C001D96AE0FBF1F0895A0915B03B0915C0384
:10362C0080915D0390915E030895E8EEF3E060E015
:10363C0070E00E946522DF01CB01BBDF6627772794
:10364C000895EC91F0E00E949821A8E0BCE481E0A0
:10365C0090E00E946522E0CFE0935B03F0935C0363
:10366C0060935D0370935E030895D6DFDECF0E94F6
:10367C006721E5E0F0E060E070E00E94E821089549
:10368C000E946721E4E1F0E060E070E00E94E0213C
:10369C0008950E946721A431E0E0BE07E0E08E07A8
:1036AC00E0E09E070895E985FA85BBDE662777275B
:1036BC000E942322D1CFE8EEF3E060E070E00895A1
:1036CC00E0E0E0932703E09328030895A92DEAE0B6
:1036DC000E94B6210E2E0895A22FE3E60E94B62179
:1036EC000895A0E0F0FCA1E0E0E00E94A221089582
:1036FC00E0E00E94BB21E0210895E0911C0391DEE3
:10370C00FF27662777270895E0E00E94A221E02199
:10371C000895ED81FE81A0916703B09168038091BB
:10372C00690390916A03662777270E94E0210E2E89
:10373C00EAE0F0E060E070E00E94E8210895E09398
:10374C004F03F09350030895EFDDAD81BE818827C0
:10375C0099270E9467210895A630E0E0BE07E0E0BB
:10376C008E07E0E09E070895A0914F03B09150039F
:10377C000895E0914F03F09150030895ED81FE817F
:10378C00A0916703B09168038091690390916A03DB
:10379C00662777270895E32FA091A303B091A40384
:1037AC008091A5039091A603FF27662777270E9497
:1037BC0019200895E32FF0E0A091A303B091A40386
:1037CC008091A5039091A6030E9498210E94192034
:1037DC00A1CD662777270E9419200E94A320089567
:1037EC00A0915103B091520308950E949D210E9413
:1037FC00BB2290CDA32FBB27E091A303F091A40390
:10380C006091A5037091A603F0CFEAE0F0E00E946E
:10381C003B220895E0914103F091420308950E2E4E
:10382C00A0911603ECE30E94B6210E220895E091BC
:10383C000B03A0E0B0E00E94EF22E0910C03A1E0AA
:10384C00B0E00E94EF22E0910D03A2E0B0E00E94F4
:10385C00EF22E0910F03A3E0B0E00E94EF22EE898B
:10386C00A4E0B0E00E94EF22EF89A5E0B0E00E9456
:10387C00EF22E88DA6E0B0E00E94EF22E091100369
:10388C00A7E0B0E00E94EF22E0911103A8E0B0E0C5
:10389C000E94EF22E0911203A9E0B0E00E94EF2217
:1038AC00E0911503AAE0B0E00E94EF2241DEA9E10D
:1038BC00B0E00E94E722EA89A4E1B0E00E94EF2286
:1038CC00EB89A5E1B0E00E94EF22EC89A6E1B0E023
:1038DC000E94EF22EE85ABE0B0E00E94EF22EF8574
:1038EC00ACE0B0E008950E94EF22E889ADE0B0E0D2
:1038FC000E94EF22ED81FE81ADE1B0E00E94E72253
:10390C00E0911A03AEE0B0E00E94EF22E0911C03BC
:10391C00AFE0B0E00E94EF22E0911B03A0E1B0E029
:10392C000E94EF22E32FA1E1B0E00E94EF22E98593
:10393C00FA85AFE1B0E00E94E722EA8DA2E1B0E0A7
:10394C000E94EF22E98DA3E1B0E00E94EF22E0910A
:10395C008F03F09190036091910370919203A1E217
:10396C00B0E00E94E21F0E94E722E0913503F09143
:10397C003603A3E2B0E00E94E722E0913903F09114
:10398C003A03A7E2B0E00E94E722E0E023FCE1E08A
:10399C00A7E1B0E00E94EF223DDFA5E2B0E00E947B
:1039AC00E7220895EAE00E94BB210E2E0895AA2D6D
:1039BC00EAE00E94B6210E2EA0E027FCA1E0E0E098
:1039CC000E94A2210E220895A0E0F2FCA1E0E0E00A
:1039DC000E94A2210E220895A82DEAE00E94B62191
:1039EC000E2E0895E0E00E94A2210E2208950E22D0
:1039FC00A22FE3E60E94A221E0210895A22FE3E684
:103A0C000E94A221E0210895E0912403EF5FE0934E
:103A1C002403E0912303A0912403EA170895A091B5
:103A2C003503B09136030895E0913503F0913603D8
:103A3C000895E0913903F0913A030895E091A303BE
:103A4C00F091A4036091A5037091A6030895A0E0E2
:103A5C00B0E080E09FE30E9453200895E09393032D
:103A6C00F093940360939503709396030895E091FB
:103A7C007303F0917403609175037091760308954C
:103A8C00EAE0F0E00E9428220895A0917303B0911F
:103A9C0074038091750390917603089525DC29CCED
:103AAC00E0936F03F0937003609371037093720350
:103ABC000895F0E0EA0FFB1FE0933303F093340317
:103ACC00AEE30C9403190E940319A0E00C940319A3
:103ADC00E0913403AE2F0E940319A09133030C9490
:103AEC000319B0E0E2E0F0E00E943B220895EAE026
:103AFC00E8AFE9AFEAAF0895A0916B03B0916C0306
:103B0C0080916D0390916E0308950E94E8210E2E12
:103B1C00F3CFAA30E0E0BE07E0E08E07E0E09E07BE
:103B2C0008957FDCEAE0F0E060E070E008950E9428
:103B3C006522DF01CB01EAE0F0E060E070E00E947A
:103B4C007F220895DF01EAE0F0E00E946D220895E3
:103B5C00A0911F03BB27EAE0F0E00E946D220895BC
:103B6C00E4E6F0E060E070E00895C6DFEAE0F0E043
:103B7C0060E070E00895A0E022FCA1E0EA2FEE0FD7
:103B8C0008950E2EA0E022FCA1E0EA2FEE0FEE0F1E
:103B9C00E00DEE8F0895A0912D03B0912E030895A2
:103BAC00E4E6F0E00E942822DF01EAE0F0E00E9467
:103BBC006A22EDAF0895DF01EAE0F0E00E946A228C
:103BCC000895EAE0F0E00E946A220895BB27EAE03B
:103BDC00F0E00E946D220895E89420F8CCCF0E946A
:103BEC004022DF01CB01EAE0F0E060E070E00E94EF
:103BFC007B22089503DCEAE0F0E060E070E00895D9
:103C0C00DF01CB01E0E0F0E060E171EC0E943621D5
:103C1C000895DF01CB01E0E0F0E066EC72EC0E946D
:103C2C0036210895DF01CB01E0E0F0EC69E774EC9C
:103C3C000E9436210895A0915703B091580308951E
:103C4C00E0E1F7E20E943B227DCFE8EEF3E00E9438
:103C5C003B2278CFE4E6F0E00E943B2273CFEAE00F
:103C6C00F0E00E946D22EFAF08953EDBE4E665CBF9
:103C7C00A0915903B0915A030895EB81FC81F695FC
:103C8C00E79508950E94282296CFA0913B03B0910E
:103C9C003C030895E0912003E170EE0FE058089585
:103CAC00E695E695E170EE0FEE0F08950E2EA0E06E
:103CBC00F199A1E0EA2FEE0FEE0FEE0F08950E0E24
:103CCC00A0E020FCA1E0EA2FE295E07FE00D089552
:103CDC00E52FF0E0DE01D096AE0FBF1F08950E94D5
:103CEC00A2210E2EAA8108950E94A2210E2AAA8139
:103CFC000895AF81B885C4CEE3E10E94A221E029EA
:103D0C000895E62DF0E0DE011D96AE0FBF1F08955D
:103D1C00A0915F03B0916003809161039091620365
:103D2C000895EC91F0E00E949821A8E0BCE481E0B9
:103D3C0090E00E946522ECCFE0935F03F093600368
:103D4C0060936103709362030895E2DF6ECCE985A2
:103D5C00FA8567DB662777270E942322EDCFA09197
:103D6C006703B09168038091690390916A03089589
:103D7C00EDABF5DFEAE0F0E060E070E0D8CEEEAB62
:103D8C00EEDFEAE0F0E060E070E00E947F22EFAB53
:103D9C0008950FDCF695E795D7CBEC8F3DDAA4367A
:103DAC00E0E0BE07089538DAE4E6F0E06BCF34DAF1
:103DBC0067CE32DA06CFE9E3E9AFE0E5EAAFEEE34E
:103DCC00EBAF0895A0913103B09132030895A09107
:103DDC003F03B09140030895E170E795E0E0E7956B
:103DEC00AE2F0895E295EF70E695E170E295E07FD5
:103DFC00EE0FEE0FEA2BAE2F0895E295EF70E695DD
:103E0C00E695E170E295E07FEE0FEA2BAE2F089578
:103E1C00E295E170E295E07FEA2BAE2F0895E17018
:103E2C00EE0FEE0FEE0FEA2BAE2F0895E695E17034
:103E3C00EE0FEE0FEA2BAE2F0895E695E695E170A6
:103E4C00EE0FEA2BAE2F0895E695E695E695E17018
:103E5C00EA2B0895E695E170E295E07FEE0FEE0F08
:103E6C00EA2BAE2F0895E695E695E170E295E07F9A
:103E7C00EE0FEA2BAE2F0895E695E695E695E170E8
:103E8C00E295E07FEA2BAE2FEE8D0895E695E69550
:103E9C00E695C5CFE295EF70E695E170EE0FEE0F6B
:103EAC00EA2BAE2F0895E295EF70E695E695E1705A
:103EBC00EE0FEA2BAE2F0895E295EF70E6958CCFBE
:103ECC00E295EF70E695E6950895E170E295E07F56
:103EDC00EA2BAE2F0895E170E295E07FEE0FEE0F26
:103EEC00EA2BAE2F0895E695E170E295E07FEE0F98
:103EFC00EA2BAE2F0895E170EE0FEA2BAE2F08954A
:103F0C00E295EF70E695E1CF289885E28A95F1F776
:103F1C0051E008955E9885E28A95F1F7ECE0E51B97
:103F2C00089585E28A95F1F75E9A85E28A95F1F714
:103F3C0008955D9A85E28A95F1F7289A84E191E0DB
:103F4C000197F1F7E1CF109639F08DEC9AE00197DB
:103F5C00F1F7A8951197C9F70895552342F45038F5
:103F6C0011F4E0FF04C03196691F791F6BF050E823
:103F7C00572711F45F93CFC05F3F31F0660F000CF1
:103F8C0057956795752F08955F9300200AF0CFC061
:103F9C00C8C050E8192E1522880F991F9527550F68
:103FAC00879550E8072E0522660F771F7527550F4A
:103FBC0067950895689401C0E8945F93F2DF7038B8
:103FCC0018F07F3F08F4A7C056E1571BAAF451958F
:103FDC0058300EF4593030F0EFEFFFEF6FEF7FE712
:103FEC0077F91AC077275523B9F0EE0FFF1F661F1C
:103FFC00771F5A95D1F710C07727583028F0EF2F3C
:10400C00F62F672F5850F9CF552331F076956795D9
:10401C00F795E7955A95D1F700200AF45BD15F919B
:10402C000895689401C0E894309760407040B1F0F6
:10403C00002426F0772312F400944CD1172E7EE145
:10404C00112032F07A95EE0FFF1F661F111CF9CF6D
:10405C00EF2FF62F612D5F938ADF5F9108954F93B9
:10406C00AF01FD01DA01AB01BC01CA01402D012CED
:10407C00142E4F910895EA0FFB1F681F0895E095C9
:10408C00F0956095EF5FFF4F6F4F08955F9381DF61
:10409C00903871F150E8152604C05F937ADF9038A0
:1040AC0039F1703821F1572F591B2BF112F4D7DF4E
:1040BC00FACF583118F0AA27BB278827583028F098
:1040CC00AB2FB82F88275850F9CF552329F0869558
:1040DC00B795A7955A95D9F7502D512572F0CBDF8E
:1040EC0038F46795F795E795739513F420C0B7DF0F
:1040FC003EDF5F910895D8F7FBCFEA1BFB0B680BF3
:10410C0051F010F40094BBDF662392F3EE0FFF1F07
:10411C00661F7A95CBF7EE27FF27662777275F91E7
:10412C000895EFEFFFEF6FE77FEF5F910895EFEFEB
:10413C00FFEF6FE77FE75F9108955F932ADF703899
:10414C0051F3903841F301240894791F23F41CF3A4
:10415C0000203AF3ECCF0F921F932F933F934F9382
:10416C00112722279927689FA0018F9F302D410D81
:10417C00591F6B9F300D411D591F8E9F27D0BF9F1C
:10418C0025D06A9F23D0BE9F1DD0AF9F1BD0AE9F62
:10419C00110D291F391F491F591FE32FF42F652FAC
:1041AC00522F4F913F912F911F910F9066232AF020
:1041BC00550FEE1FFF1F661F02C073954BF2CDDE2D
:1041CC005F910895100D211D391F02C0200D311D66
:1041DC00491F591F08955F93DCDE703821F41120BC
:1041EC000AF49FCFA4CF903809F495CF01240894FA
:1041FC00970B1BF4D4F30020F3CF792F1F932F933D
:10420C003F934F93112411272227332744275527F7
:10421C0090E2AE17BF078607410730F0AE1BBF0B0D
:10422C00860B410B089401C08894551F221F331F25
:10423C00111CAA1FBB1F881F441F9A9551F7F90127
:10424C00612D4F913F912F911F91662332F0550FA5
:10425C00EE1FFF1F661F7A9543F27FDE5F91089574
:10426C0099239AF0772342F0971748F029F4AE1768
:10427C00BF07860720F031F098948894089598949D
:10428C00089408951894889408957723C2F7971783
:10429C0098F3A9F7EA17FB07680788F399F3ECCFB3
:1042AC00DFDFE1E009F008F0EE270895D9DFE1E067
:1042BC0009F008F4EE270895EA0FFB1F681F791F19
:1042CC000895AE1BBF0B860B970B0895F195E195E6
:1042DC00F0400895F09560957095E195FF4F6F4F04
:1042EC007F4F0895EE230E2EEA2F19F0E6950A94CF
:1042FC00E9F70895EE230E2EFD0121F0F695E795D2
:10430C000A94E1F70895F695E795F695E795F695F5
:10431C00E795F695E7950895FE2FFF0FFF0B6F2F8E
:10432C007F2F08956F2F660F660B762F08958B2FB6
:10433C00880F880B982F0895EA17E1E009F0EE2713
:10434C000895AE17E1E00CF4EE270895AE17E1E006
:10435C000CF0EE270895EA17E1E00CF0EE27089533
:10436C00AE17E1E008F0EE270895EA17E1E008F057
:10437C00EE270895EA17FB07E1E009F0EE27089510
:10438C00AE17BF07E1E008F4EE270895AE17BF079C
:10439C00E1E008F0EE270895EA17FB07E1E008F0EA
:1043AC00EE270895EA17FB0768077907E1E009F0A3
:1043BC00EE270895AE17BF0786079707E1E00CF0CC
:1043CC00EE270895EA17FB0768077907E1E00CF080
:1043DC00EE270895FA9FF02DEB9FF00DEA9FE02D4C
:1043EC00F10D08957A9F702D6B9F700DF89F700DD5
:1043FC00E99F700D6A9F602D710DFB9F600D711D03
:10440C00E89F600D711D8827FA9FF02D610D781FB4
:10441C00EB9FF00D611D781FEA9FE02DF10D681FD9
:10442C00781F08956E2F6A9FF0016B9FF00D089511
:10443C0074D0D0DF0EF44ADF08957DD0D3DF0EF4B4
:10444C0049DF08950024112490E1AA0FBB1F001C22
:10445C00111C0E1A1F0A18F40E0E1F1E01C0A160AB
:10446C009A9599F7FD01D001089557D0EBDF0EF422
:10447C002DDF08953F934F935F930024112444271D
:10448C00552730E2AA0FBB1F881F991F001C111C57
:10449C00441F551F0E1A1F0A460B570B28F40E0EFD
:1044AC001F1E461F571F01C0A1603A9559F7FD0109
:1044BC00BC01D001CA015F914F913F9108953BD04F
:1044CC00D9DF0EF407DF0895BDDFFD010895E894F0
:1044DC00B7FF04C0A095B09511966894F7FDF6DE71
:1044EC00B1DFFD010EF4F2DE0895C4DFFD01BC0165
:1044FC000895E89497FF09C0A095B0958095909584
:10450C00AF5FBF4F8F4F9F4F689477FDE3DEB2DFF5
:10451C00FD01BC010EF4DEDE0895E894F7FF02C045
:10452C00D5DE6894B7FF06C0A095B095119600F83B
:10453C00039400FA0895E89477FF02C0CBDE6894E8
:10454C0097FF0BC00024A095B0958095909511967F
:10455C00801D901D00F8039400FA0895ED93FD93CF
:10456C006D937C930895689401C0E89401D05CDD50
:10457C00182E862F612D192E972F712D1B2EBF2FC4
:10458C00F12D1A2EAE2FE12D0895129602D0BF01F7
:10459C001297119602D0FE2F1197F999FECFFF9327
:1045AC00FFB7F894A1BDB2BDF89AE0B5FFBFFF917B
:1045BC00089507D012960F01FB0103D0F00112975A
:1045CC00089507D01196EF93EF2F03D0EF91119729
:1045DC000895F99B02C0A895FCCF9FB7F894A1BD94
:1045EC00B2BDF89A80B5E81719F0E0BDFA9AF99ABD
:1045FC009FBF089500240E160F06060607060895A1
:10460C0000240A160B06089500240A160B06080649
:10461C0009060895EA17FB07680779070895AE178E
:10462C00BF07860797070895E894EE2309F068946E
:10463C000895AC0FBD1F05900D928A95E1F7089572
:00000001FF
